:0A000000A001A101A2018A11952FB1
:100F1400830121080319A203A103210A0319220A48
:100F2400031908008A2F831203179E0183160313E3
:100F3400870183128701013087009830A1003A307D
:100F4400A2008A27023087009830A1003A30A2001C
:100F54008A27043087009830A1003A30A2008A27FB
:100F6400083087009830A1003A30A2008A27103058
:100F740087009830A1003A30A2008A2720308700E9
:100F84009830A1003A30A2008A2740308700983078
:100F9400A1003A30A2008A27803087009830A1004F
:100FA4003A30A2008A27403087009830A1003A30B6
:100FB400A2008A27203087009830A1003A30A2008E
:100FC4008A27103087009830A1003A30A2008A277F
:100FD400083087009830A1003A30A2008A270430F4
:100FE40087009830A1003A30A2008A270230870097
:0C0FF4009830A1003A30A2008A279D2FFF
:00000001FF
